:100000008C28640011200318012842200830A30026
:1000100043201120A20C0C28A30B082843202208FF
:10002000080036088400340884178004841300050F
:1000300033193406FF3E0800A60036088400093054
:10004000A70003102820A60CA70B22280314282899
:100050008413B31D372800083404331D3406800090
:10006000841700083404031C340680004328000869
:100070003404031C34063319340680008417340911
:10008000800543283317330D0639A0005120A10005
:10009000A00A5120331F6B283313A00002308220A6
:1000A0006B2800308A00200882070134753403343D
:1000B000153400343C340C34D934A301A200FF3091
:1000C000A207031CA307031C87280330A100DF300D
:1000D0006B205F28A101E83EA000A109FC30031CB1
:1000E0007428A00703187128A0076400A10F7128C5
:1000F00020187A28A01C7E2800007E280800031003
:10010000A10CA00CFF3E03187F282008872883132A
:10011000031383126400080064308A015D200630F6
:10012000B6004030B4000430B3008A010120B800AA
:10013000061483160610323083128A015D200610E1
:1001400083160610323083128A015D200630B60015
:100150008030B4000430B30038088A011C208A01C2
:080160008F2863008A01B12819
:02400E00713F00
:00000001FF
